:1000FB007F061170D2AFD288D2A8E4FFFED2B70F21
:10010B00BF00010EBE75F6BF30F3E4FEFFC3EF94E4
:0F011B0030EE947550E4C2B70FBF00010E80EEB6
:10007000EF14B40800503A90008125E05002058347
:1000800073019101950199019D01A101A501A901AA
:10009000AD7E40801E7EA0801A7ED080167EE880D5
:1000A000127EF4800E7EFA800A7EFD80067EFF803E
:1000B000027ED07598507589217588408E8D8E8B03
:0900C000758780C298C299D28EA6
:0100C9002214
:06012A0074082EF8E6FF48
:080130008F993099FDC299225C
:02000B00010DE5
:07000D00C0E0C0D075D01067
:10001400758CFD758A1EE50CC39403502CE50BC347
:100024009408501E050B7408250CF8C010E625E052
:10003400D010F67408250CF8E6FFA2B2E4334FF6AC
:100044008025050C750B00801EC28CC2A9E509F43D
:100054006013E50AF4600E7E0112012A12012A31AE
:070064002A0EBE03F4D2A82E
:05006B00D0D0D0E0320E
:0200030001CA30
:1000CA00C0E0C0D075D010C2ACC2A8D2A9758CFD50
:1000DA00758A1E750C007408250CF87600050CE567
:1000EA000CB403F2750C00750B00D28CD0D0D0E0A2
:0100FA0032D3
:03000000020138C2
:0C013800787FE4F6D8FD7581170200FB0B
:00000001FF
